:08000000D2C546C792C7FCCF30
:1000080069C8FACF4BC8F8CFF7CFA7C7F5CFF4CF59
:10001800F3CFF2CFF1CFF0CFEFCFEECFEDCF00009F
:1000280000000000000000000000000000000000C8
:1000380000000000000000000000000000000000B8
:1000480000000000000000000000000000000000A8
:100058000000000000000000000000000000000098
:100068000000000000000000000000000000000088
:100078000000000000000000000000000000000078
:100088000000000000000000000000000000000068
:100098000000000000000000000000000000000058
:1000A8000000000000000000000000000000000048
:1000B8000000000000000000000000000000000038
:1000C80000000000000000FFFFFFFFFFFFFFFFFF31
:1000D800FFFFFFFFFEFEFEFEFEFEFEFEFEFEFEFE34
:1000E800FE0000000000000000000000000000000A
:1000F80000000000000000000000000000000000F8
:1001080000000000000000000000000000000000E7
:1001180000000000000000000000000000000000D7
:1001280000000000000000000000000000000000C7
:1001380000000000000000000000000000000000B7
:1001480000000000000000000000000000000000A7
:100158000000000000000000000000000000000097
:100168000000000000000000000000000000000087
:100178000000000000000000000000000000000077
:100188000000000000000000000000000000000067
:100198000000000000000000000000000000000057
:1001A8000000000000000000000000000000000047
:1001B8000000000000000000000000000000000037
:1001C80000000000000000000000000010101010E7
:1001D8001010100000100000002424480000000047
:1001E8000000000000002828FE2828FE282800001B
:1001F8000000087C8A8890907C121222A27C200041
:1002080044A848101020204048948800007088882E
:10021800889060908A848A70000020204000000046
:100228000000000000000010202040404040202036
:100238001010000010080804040404080810100036
:100248000010925438549210000000000000001072
:100258001010FE1010100000000000000000000048
:10026800000000301020000000000000FE00000028
:100278000000000000000000000000000000303016
:100288000000040808101020204040808000007CF6
:1002980086828A829282A282C27C0000103010106C
:1002A8001010101010103800007C8202020204089E
:1002B800102040FE0000FE0408103C0202020282E8
:1002C8007C0000040C1424448484FE04040400000C
:1002D800FE8080FC0202020202827C00007C828096
:1002E80080FC82828282827C0000FE020204081066
:1002F800202020202000007C828282443844828290
:10030800827C00007C828282827E020202827C00E1
:100318000000003030000000003030000000000015
:1003280030300000000030102000000204081020C7
:1003380040201008040200000000007E0000007E3B
:1003480000000000008040201008040810204080B1
:10035800000038448202020408101000100000381F
:10036800448202027A8A8A8A8A7C0000384482821D
:10037800828282FE8282820000FC828282FC8282E9
:10038800828282FC00007C828080808080808082E3
:100398007C0000F8848282828282828284F8000053
:1003A800FE808080FC8080808080FE0000FE80804F
:1003B80080FC80808080808000007C8280808080BB
:1003C800808E82827E00008282828282FE82828287
:1003D8008282000038101010101010101010380011
:1003E800000E0404040404040404847800008488CF
:1003F80090A0C0A090888482820000808080808045
:100408008080808080FE000082C6AA9292928282BA
:10041800828282000082C2A2A29292928A8A8682F4
:1004280000007C8282828282828282827C0000F842
:100438008482828284F880808080000038448282AE
:10044800828282828A443A0000F88482828284F816
:100458009088848200007C828080807C02020282F4
:100468007C0000FE1010101010101010101000006A
:1004780082828282828282828244380000828282E0
:10048800828244442828101000008282829292922C
:1004980092929254280000828244442810284444AE
:1004A800828200008282444428101010101010002C
:1004B80000FE020404081020404080FE00000000F6
:1004C8000000000000000000000000000000000024
:1004D8000000000000000000000000000000000014
:1004E8000000000000102828444482820000000018
:1004F800000000000000000000000000FE000004F2
:100508000400000000000000000000998181003C08
:10051800A5A5A53C00818164000000000000000042
:1005280000000000000000000000000000000000C3
:1005380000000000000000000000000000000000B3
:1005480000000000000000000000000000000000A3
:100558000000000000000000000000000000000093
:100568000000000000000000000000000000000083
:100578000000000000000000000000000000000073
:100588000000000000000000000000000000000063
:100598000000000000000000000000000000000053
:1005A8000000000000000000000000000000000043
:1005B8000000000000000000000000000000000033
:1005C8000000000000000000000000000000000023
:1005D8000000000000000000000000000000000013
:1005E8000000000000000000000000000000000003
:1005F80000000000000000000000000000000000F3
:1006080000000000000000000000000000000000E2
:10061800000000000000000000000000000000884A
:10062800888888888850502000000000000000005A
:1006380000000000000000000000000000000000B2
:1006480000000000000000000000000000000000A2
:100658000000000000000000000000000000000092
:100668000000000000000000000000000000000082
:100678000000000000000000000000000000000072
:10068800000000000000000060920C000000000064
:100698000000000000000000000000000000004012
:1006A800A0401C2220202020221C00040EE4000070
:1006B80044FE82828282FE001C94D49494D4141C3A
:1006C8001C1C363E1C00000000000000000000005A
:1006D8000000000000000000000000000000000012
:1006E8000000000000000000000000000000000002
:1006F80000000000000000000000000000000000F2
:1007080000000000000000000000000000000000E1
:10098800000000000202000684C4A494948C840031
:10099800000000000000000000000000000000004F
:1009A800000000000000000000000000000000003F
:1009B800000000000000000000000000000000002F
:1009C800000000000000000000000000000000001F
:1009D80000000000000000000000000000000038D7
:1009E800448282828282FE8282820000FE8080802F
:1009F800FC8282828282FC0000FC828282FC8282EB
:100A0800828282FC0000FE808080808080808080DE
:100A18008000007E2222222222424282FE820000A0
:100A2800FE808080FC8080808080FE000092929210
:100A380092527C529292929200007C8202023C0274
:100A4800020202827C000082868A8A929292A2A284
:100A5800C282003882868A8A929292A2A2C28200B8
:100A680000848890A0C0A0908884828200007E22A2
:100A780022222222222222A242000082C6AA929286
:100A880092828282828200008282828282FE8282B6
:100A980082828200007C8282828282828282827C3E
:100AA8000000FE828282828282828282820000F834
:100AB8008482828284F88080808000007C828080AA
:100AC8008080808080827C0000FE10101010101042
:100AD8001010101000008282828242221408102016
:100AE8004000007C92929292927C101010100000AC
:100AF80082824444281028444482820000848484EA
:100B0800848484848484FEFD020082828282827EC0
:100B180002020202020000929292929292929292A1
:100B280092FE0000929292929292929292FE02000B
:100B380000C04040407844424242447800008282EB
:100B4800828282F28A8A8A8AF20000404040407893
:100B580044424242447800007C820202023E020281
:100B680002827C00009CA2A2A2A2E2A2A2A2A29C53
:100B780000003E42828282423E12224282000000EF
:100B88000E00000000000000000001000200860BBB
:100B98000100D701880B080006008A0B0000F894B2
:100BA800EE27ECBBF1E0FBBFEBBFE5BFF8E1F1BD21
:100BB800E1BD8DE0A2E0BB27ED938A95E9F780E0DF
:100BC80094E0A0E6ED930197E9F7E2E9FBE085916F
:100BD8009591009761F0A591B59105901590BF0189
:100BE800F00105900D920197E1F7FB01F0CFEFE5D9
:100BF800EDBFE4E0EEBFC0E6D1E073C2E89422F8AE
:100C080022FEFECFE0E09199E1E01E2EE72DA1E063
:100C18002CD5E095E12111F4919801C0919AE0E07A
:100C28008999E1E01E2EE72DA1E01FD5E12911F4F5
:100C3800899801C0899A88EA97E00197F1F7E0E07E
:100C48008999E1E01E2EE72DA1E00FD5E095E1217D
:100C580011F4899801C0899A84E091E00197F1F72D
:100C6800E0E08199E1E01E2EE72DA1E0FED4E1212C
:100C780044D521F880E293E00197F1F7E0E081990B
:100C8800E1E01E2EE72DA1E0B0E0F7D4A12DB0E001
:100C9800EA23FB23309711F4689421F884E393E066
:100CA8000197F1F7E0E021FCE1E008952BD500E0A1
:100CB800E89422F822FEFECF10E01830A8F5E0E014
:100CC8008999E1E01E2EE72DA1E0CFD4E12911F4A6
:100CD800899801C0899A85E38A95F1F7E0E08999B6
:100CE800E1E01E2EE72DA1E0C0D4E095E12111F44A
:100CF800899801C0899A85E18A95F1F70695E0E01F
:100D08008199E1E01E2EE72DA1E0B0E0B6D4A12D37
:100D1800B0E0EA23FB23309709F0006888EF90E001
:100D28000197F1F71F5FC9CFE02FEFD40895AA9379
:100D38001A93E89422F822FEFECF10E0183008F04B
:100D480045C0E0E08999E1E01E2EE72DA1E08DD4B1
:100D5800E12911F4899801C0899A85E38A95F1F708
:100D6800E981E17071F0E0E08999E1E01E2EE72D5C
:100D7800A1E07BD4E095E12111F4899801C0899A1A
:100D88000CC0E0E08999E1E01E2EE72DA1E06DD4CA
:100D9800E12911F4899801C0899AE981E695E983E6
:100DA80088EC90E00197F1F7E0E08999E1E01E2EE8
:100DB800E72DA1E05AD4E095E12111F4899801C00A
:100DC800899A8BE08A95F1F71F5FB8CF18815AC0CE
:100DD80015DFACECACDFAEEBAADF68DF9E2E66DF7A
:100DE8006E2E0CDFACECA3DFA4E4A1DF67FE0EC01F
:100DF800992029F4E62DE095EF5F6E2E01C06094EE
:100E0800E92DE095EE5F9E2E689401C0E89420F8E5
:100E1800A62DB0E0E0E0F1E04AD4DF01E92DF0E0F2
:100E2800EA0FFB1F2F01F201AAE0B0E038D42ED45C
:100E38002F01F2010895BA93AA93E0E3CE2EE0932E
:100E4800B401A881B981A436E0E0BE0740F0E8818A
:100E5800F981E456F040E883F983C394F2CFA8817E
:100E6800B9811A9758F0E881F9813A97E883F983AC
:100E7800E091B401EF5FE093B401F1CFE881E05D68
:100E8800E093B50122960895AA93EA93FA93EFB7EF
:100E9800EA93E0E0E4BDE82DF0E0309711F4E8EAE9
:100EA8000BC0E130A0E0FA0711F4E0EA05C0E23037
:100EB800A0E0FA0711F4E7E8E2BFEDE0BE1630F46F
:100EC800E8B7E160E8BFE9B7E16024C0EBB7EF7BC2
:100ED800EBBF8394E82DF0E0E130A0E0FA0729F4B5
:100EE800E2EDF0E0FBBDEABD16C0E230A0E0FA0793
:100EF80029F4E0EFF0E0FBBDEABD0DC0E330A0E06F
:100F0800FA0749F4E9B7EF7EE9BFEBB7EF7BEBBF30
:100F1800E9B7EE7FE9BFE991EFBFF991E991A991AE
:100F28001895EA93FA93EFB7EA93E0E0F0E0FDBD95
:100F3800ECBDE4BDE8B7E061E8BFE9B7E061E9BF4F
:100F4800E4EBF0E0FBBDEABD8824BB24689422F8FA
:100F5800E991EFBFF991E99118950A921A92AA932B
:100F6800BA93EA93FA93EFB7EA93CCD3E9B7EE7F53
:100F7800E9BFE82DF0E0309749F5E1E0EEB9C29815
:100F8800E0916001ADE0EA9FF001EA5DFF4FDF010B
:100F9800EB2DF0E0EA0FFB1F049110E01E3198F4EE
:100FA8000FB9E12FF0E0EF59FE4FE081ADE0EA9F85
:100FB800F001EA5DFF4FDF01EB2DF0E0EA0FFB1FC8
:100FC80004911F5FEBCF779BFECF59C0E130A0E0C3
:100FD800FA0749F5E0E0EEB9C298E0918001ADE08A
:100FE800EA9FF001EA5DFF4FDF01EB2DF0E0EA0F29
:100FF800FB1F049110E01131A8F40FB9E12FF0E0C4
:10100800EF57FE4FE081ADE0EA9FF001EA5DFF4F48
:10101800DF01EB2DF0E0EA0FFB1F0491779BFECF79
:101028001F5FE9CF2CC0E230A0E0FA0749F5E0E005
:10103800EEB9C298E091A001ADE0EA9FF001EA5D47
:10104800FF4FDF01EB2DF0E0EA0FFB1F049110E0EA
:101058001F30A8F40FB9E12FF0E0EF55FE4FE08103
:10106800ADE0EA9FF001EA5DFF4FDF01EB2DF0E014
:10107800EA0FFB1F0491779BFECF1F5FE9CFC29A4F
:10108800B394E9B7EE7FE9BF40D3E991EFBFF99197
:10109800E991B991A991199009901895EA93EFB738
:1010A800EA93BB24EAB7E064EABFEBB7E064EBBFBE
:1010B800E991EFBFE9911895AA93E881E06EE7B945
:1010C80085E38A95F1F7369A349BFECF349AE5B1D9
:1010D80021960895EA93EFB7689422F8EFBFE99153
:1010E8001895E3E0E8BBECE2E7BBE0E0E5BBE4BB76
:1010F800E0ECE2BBE1E1E1BBE1E0E3BFE0E0E2BF5D
:10110800EFBDE6E0EEBDE0E0EDBDECBDE7BDE6BD60
:10111800E4E6F0E0FBBDEABDE0E0E9BDE8BDE2BD24
:10112800E7E0E5BDE0E0E4BDE3BDEBB7E06CEBBFB5
:10113800EAE0E5BFE0ECEABFE0E5E9BFE0E0EAB9F4
:10114800E0E8E8B9E0E0E0BFE0EEE7B9E6E8E6B9F4
:10115800E0E0E8BBEFEFE7BBE4E5EDB9E1E0EEB9CD
:10116800E0E0E6BF789422FE6FC22197E89422F867
:10117800A091D601AF5FA093D601A150E091D7010D
:10118800AE1708F493C0E0E0E093D601E091D701F0
:10119800F0E0A091B601B091B7018ED2E093C601FC
:1011A800F093C701E0E0E093B601E093B701A091A6
:1011B800B801B091B901E091D701F0E07DD2E09398
:1011C800C801F093C901E8EBF1E0A0E0B0E0A0832A
:1011D800B183A091BA01B091BB01E091D701F0E0D1
:1011E8006BD2E093CA01F093CB01EAEBF1E0A0E007
:1011F800B0E0A083B183A091BC01B091BD01E091A2
:10120800D701F0E059D2E093CC01F093CD01ECEB9B
:10121800F1E0A0E0B0E0A083B183A091BE01B0915D
:10122800BF01E091D701F0E047D2E093CE01F093FF
:10123800CF01EEEBF1E0A0E0B0E0A083B183A09194
:10124800C001B091C101E091D701F0E035D2E0933F
:10125800D001F093D101E0ECF1E0A0E0B0E0A08390
:10126800B183A091C201B091C301E091D701F0E030
:1012780023D2E093D201F093D301E2ECF1E0A0E0B5
:10128800B0E0A083B183A091C401B091C501E09101
:10129800D701F0E011D2E093D401F093D501E4EC4A
:1012A800F1E0A0E0B0E0A083B18368C0A0E004DF73
:1012B800F0E0A091B601B091B701EA0FFB1FE093EF
:1012C800B601F093B701A1E0F7DEF0E0A091B80114
:1012D800B091B901EA0FFB1FE093B801F093B9018F
:1012E800A2E0EADEF0E0A091BA01B091BB01EA0FFA
:1012F800FB1FE093BA01F093BB01A3E0DDDEF0E051
:10130800A091BC01B091BD01EA0FFB1FE093BC01A5
:10131800F093BD01A4E0D0DEF0E0A091BE01B09151
:10132800BF01EA0FFB1FE093BE01F093BF01A5E0E8
:10133800C3DEF0E0A091C001B091C101EA0FFB1F2C
:10134800E093C001F093C101A6E0B6DEF0E0A09101
:10135800C201B091C301EA0FFB1FE093C201F093F1
:10136800C301A7E0A9DEF0E0A091C401B091C501D6
:10137800EA0FFB1FE093C401F093C501A0E0B09908
:10138800A1E0A03029F0A0E025FCA1E0A03009F000
:101398000DC0A0E0B099A1E0A03029F0A0E025FCA4
:1013A800A1E0A03009F002C0689425F8A0E0B09947
:1013B800A1E0A03029F4A0E025FCA1E0A03009F4C8
:1013C80007C0E89425F8D394E2E0ED1508F4DD248D
:1013D800E1E3AE1610F4A39403C0AA24689423F89A
:1013E800E0E0E883A881AA3150F4E881F0E0E05A0F
:1013F800FE4FA0E2A083E881EF5FE883F3CFE0E04F
:10140800E883A881A13150F4E881F0E0E058FE4F6C
:10141800A0E2A083E881EF5FE883F3CFE0E0E88310
:10142800A881A03150F4E881F0E0E056FE4FA0E238
:10143800A083E881EF5FE883F3CFE0E2E093600107
:10144800A091C601B091C701F6DCE0E3EC1510F4F9
:10145800C0926101E091B401E0936201ECE2E09393
:101468006301E091B501E0936401E6E7E09365016B
:10147800E0E2E0936601E0936701A091C801B091B2
:10148800C901D9DCE0E3EC1510F4C0926801E091E1
:10149800B401E0936901ECE2E0936A01E091B501DF
:1014A800E0936B01E6E7E0936C01E0E2E0936D0105
:1014B800E0936E01A091CA01B091CB01BCDCE0E3DE
:1014C800EC1510F4C0926F01E091B401E093700143
:1014D800ECE2E0937101E091B501E0937201E6E777
:1014E800E0937301E0E2E0937401E0937501A09149
:1014F800CC01B091CD019FDCE0E3EC1510F4C09273
:101508007601E091B401E0937701ECE2E093780191
:10151800E091B501E0937901E6E7E0937A01A091C3
:10152800CE01B091CF0187DCE0E3EC1510F4C09256
:101538008001E091B401E0938101ECE2E093820143
:10154800E091B501E0938301E6E7E0938401E0E2EE
:10155800E0938501A091D001B091D1016CDCE0E36A
:10156800EC1510F4C0928601E091B401E093870174
:10157800ECE2E0938801E091B501E0938901E6E7A8
:10158800E0938A01E0E2E0938B01A091D201B0914F
:10159800D30151DCE0E3EC1510F4C0928C01E0912A
:1015A800B401E0938D01ECE2E0938E01E091B50186
:1015B800E0938F01E6E7E0939001E1E8E093A00172
:1015C800A091D401B091D50136DCE0E3EC1510F41C
:1015D800C092A101E091B401E093A201ECE2E09392
:1015E800A301E091B501E093A401E6E7E093A5012A
:1015F800E0E2E093A601E093A701E2E8E093A80106
:10160800D20119DC20FE08C0E0E024FCE1E0F0E0B3
:10161800E755FE4FADE2A083E0E3EC1520F4C0925D
:10162800AA01E89401C0689424F8E091B401E09319
:10163800AB01ECE2E093AC01E091B501E093AD01C0
:10164800E0E8E093AE01219623FE09C0E89423F870
:10165800BFDB2F01949B02C0949801C0949A83CD5C
:10166800FFCFF195E195F0400895EE230E2EEA2F75
:1016780019F0EE0F0A94E9F70895EE230E2EFD01F6
:1016880021F0EE0FFF1F0A94E1F70895F695E7950C
:10169800F695E795F695E795F695E7950895FA9FF7
:1016A800F02DEB9FF00DEA9FE02DF10D089517D076
:1016B800F6DF0EF4D6DF08950024112490E1AA0F76
:1016C800BB1F001C111C0E1A1F0A18F40E0E1F1E39
:1016D80001C0A1609A9599F7FD01D0010895E89499
:1016E800F7FF02C0BEDF6894B7FF06C0A095B095AB
:1016F800119600F8039400FA0895E894EE2309F08F
:10170800689408951A930A93089509911991089570
:00000001FF
